:020000020000FC
:10000000DDC949C20000000025C000004FC100004A
:10001000000052C1000000000000000002030406BE
:10002000080C101820304060800002030406080C01
:10003000101820304080FF000406080C10182030F3
:10004000406080A0C0000D0D0405060D050D0603DF
:10005000030302004FB662FD1EC070FF1AC165FDAA
:10006000FAC00994C0919700C395C0939700C5E06A
:10007000C519B8F3D0919700CD1B98F3C8E7089441
:1000800083FDC795C4BDC52DCC2321F4C0E083FDFD
:10009000C0E8C4BD09C171FF03C09598AC98C09871
:1000A000C52D089483FDC795C4BDC09399006B7F8F
:1000B000C52DCF3F09F443C0C0919800C395C093AC
:1000C000980070FF37C082FD05C09598AC98C09825
:1000D0004FBE18957860C091A000CC2391F0C091DC
:1000E0009800CA95D091A000CD1B58F0777FC091A1
:1000F0009800D0919F00CD1B08F41CC0209298005E
:1001000019C09598AC98C098C5E0CA95F1F7C09110
:100110007500CA95C2FD09C0C1FD05C095FFAB9829
:1001200095FD94980EC0AD980CC095FF949895FDE0
:10013000AB9807C09598AC98C0984FBE1895209280
:1001400099004FBE1895A5C0552021F095FF959AAE
:1001500095FDC09AAC989DC0552009F0AC9A95FFCA
:10016000C09895FD959895C0552021F095FFC09AAF
:1001700095FD959A95FF959895FDC0988AC095FF35
:10018000949A95FDAB9A95FFAB9A95FD949AC5E02C
:10019000CA95F1F7552021F095FF959A95FDC09AE3
:1001A000AC9877C095FF949A95FDAB9AAD9AC5E04F
:1001B000CA95F1F7552021F095FF959A95FDC09AC3
:1001C000AC9867C0AD9A95FF949A95FDAB9AC5E03F
:1001D000CA95F1F7552009F0AC9A95FFC09895FDA6
:1001E000959857C0AD9A95FFAB9A95FD949AC5E046
:1001F000CA95F1F7552009F0AC9A95FFC09895FD86
:10020000959847C095FFAB9A95FD949AAD9AC5E035
:10021000CA95F1F7552021F095FFC09A95FD959A62
:1002200095FF959895FDC09834C095FFAB9A95FDC4
:10023000949A95FF949A95FDAB9AC5E0CA95F1F70B
:10024000552021F095FFC09A95FD959A95FF9598B8
:1002500095FDC0981EC082FF1CC0C0917500C2FDF4
:100260000BC0C1FD11C095FF949A95FDAB9A95FF07
:10027000AB9A95FD949A0DC0C1FDF5CF95FF949A68
:1002800095FDAB9AAD9A05C0AD9A95FFAB9A95FDD9
:10029000949AC52DC095089483FDC795C4BDC0939D
:1002A00099002092970064604FBE18954FB6C0E148
:1002B000C8BF6E7F4FBE18953FB68F7EABB7A07498
:1002C000A2118061A0E0ABBFA9B7AE7FA9BF7894AF
:1002D000A0916600AA2349F0A92FAF7151F1A09116
:1002E0006600AA95A093660024C040E050E0A0B349
:1002F00096FDA095A2FD4FEF96FFA3E096FDA2E02C
:10030000A5BFAA27A064AABF8D7FA0B396FDA09524
:10031000A2FD5FEF451749F7A8E161FDA0936600D4
:10032000A92FAF7119F0A8E1A093660040938D004A
:100330008160A0916700AA2331F0A0916700AA957F
:10034000A093670007C0A92FAF7121F08061AA2791
:10035000A064AABF80FF4BC0A0918D004A2F8E7F62
:10036000A92FAF71E1F0A091AE00A430C1F4403FDD
:1003700008F040EFA42FA295AF704A0F5091B00043
:10038000533069F0A695A69550FD01C0A69552FD83
:1003900003C0A41B4A2F03C04A0F08F44FEF409339
:1003A000610071FF08C0A091610050919200A517F3
:1003B00010F0509361004091AE00443029F5A091B7
:1003C000610040916300A41B70F04091CF00A40B2A
:1003D00050F0A0916300A40FA093630040F4AFEF2E
:1003E000A093630004C0A0916100A09363004091BA
:1003F0006300A09192004A1708F04A2FA091940040
:100400004A1708F04A2F542EA52DA03408F0686032
:10041000A0916000A395A093600051F0F894A9B753
:10042000A160A9BF84FF02C0A0E4ABBF3FBE189586
:1004300041E050916600552331F0A92FAF7119F4B6
:100440005A9550936600A0918D00A13018F020922B
:1004500090000DC02092910020929A00A0919000EF
:10046000AF5FA093900018F0AFEFA0939000A09121
:100470009300A65F20F05FEF5093930002C0A0931B
:100480009300F894A9B7A160A9BF84FF02C0A0E4BB
:10049000ABBF3FBE18953FB64CB55DB58F7EABB7D1
:1004A000A074A2118061A0E0ABBFA9B7AE7FA9BFC5
:1004B000789481FD26C096FFA2E096FDA3E0A5BF3B
:1004C0008260A0B396FDA095A2FF05C04093640092
:1004D0005093650033C196FFA3E096FDA2E0A5BF4F
:1004E000AA27A064AABF8D7FA92FAF7109F417C1F5
:1004F00040E0A0B396FDA095A2FD11C140938D00F0
:1005000004C196FFA3E096FDA2E0A5BF8D7F61FF29
:100510006BC096FFA2E096FDA3E0A5BFAA27A0644A
:10052000AABF82604093880050938900A090860003
:100530004A19B09087005B09BB24A2E0EA2EA22CE6
:10054000483CA0E05A0730F4A0E1BA2EE22CAAE021
:10055000AA2E27C04836A1E05A0730F4A8E0BA2EE8
:10056000E22CAFE0AA2E1DC0403DA2E05A0730F4B5
:10057000A4E0BA2EE22CAEE1AA2E13C0403AA5E0C8
:100580005A0730F4A2E0BA2EE22CACE3AA2E09C03E
:100590004839A8E05A0728F4A1E0BA2EE22CA8E7CF
:1005A000AA2EC42EA0918A00CA1AD52EA0918B0023
:1005B000DA0ADD202AF4AFEFC094D094CA1ADA0A1E
:1005C00020928C00CA14DE0418F4A1E0A0938C00E1
:1005D00040938A0050938B0040918800509189008D
:1005E0004093860050938700A09164004A1BA0911D
:1005F00065005A0B94FD7CC093FD7AC092FD76C0D5
:100600005695479591FD72C05695479590FD6EC0E1
:10061000D52EC42ED694C79461FD0CC0AC2DAC5120
:10062000AD2DA24008F07BC0DD2021F4AC2DA85CEC
:1006300008F475C0A0E0EA2E97FD08C0E090C20063
:10064000A091B400A33011F4E090CA00AAEFEA0E22
:10065000F22CF21CCE18DF084FB74170A091B40005
:10066000A330A9F4442329F095FD11C0F8949062B9
:1006700004C095FF0CC0F8949F7D9598AC98C098E5
:10068000949AAD9AAB9A71FD01C060687894442346
:1006900069F0A091B400A33031F4AFEFC094D094CE
:1006A000CA1ADA0A03C040E050E022C0A091B400A8
:1006B000A33049F4CC0CDD1CA5E0CA1AD20818F40A
:1006C000A0E0CA2ED22CAFEFCA16D20418F04FEF1A
:1006D00050E00EC0F090A700CF9C412D000C441FAD
:1006E00050E008F012C04FEF50E00FC0569547950C
:1006F00094FF07C0552309F04FEFA42FA6954A0F8A
:10070000521D4F3F520508F04FEF40938D0081601E
:1007100061FF05C0AFE1A095A923AB299A2FA8E1FD
:10072000A0936600A92FAF7119F4AAE0A093660008
:1007300061FD04C0A92FAF7109F08F7EA6E0A093E0
:100740006700A92FAF7119F4AAE0A0936700F8948D
:10075000A9B7A160A9BF84FF02C0A0E4ABBF3FBEA0
:10076000189511E00AC013E008C01AE006C01EE1A7
:1007700004C014E602C018EC00C005E1BB27BA951E
:10078000F1F70A95D9F71A95C1F708952AE338E7E2
:1007900009C020E33CE806C02AE234EB03C025E2AE
:1007A00038EC00C0652CB1E05B2E12E095FD9F7D1A
:1007B00095FF9062BB27AD9ABA95F1F7552009F0E5
:1007C000AC9ABA95F1F7AC98BA95F1F7AD98BA959D
:1007D000F1F7552021F095FF959A95FDC09AB091BB
:1007E000A800BA95F1F795FF959895FDC098B7E8E0
:1007F000BA95F1F71A95D1F6022FB22FBA95F1F703
:100800000A95D9F73A9571F6AD9A562C0895221BA0
:1008100039E0001F3A9509F40895221F211B18F4AE
:10082000210F8894F6CF0894F4CF622C722CB0E09C
:100830008894B395221F331FE0F737952795889446
:10084000912E802E020B130B10F4192D082D10F48D
:10085000889401C00894661C771CBA9571F7172D0F
:10086000062D0895322D11232AF43A9500951095FE
:10087000031B130BF894029F712C002D129F912CD7
:10088000802C7894780C172D921C292DB4E06B2EB7
:100890002695179507956A94D9F7332321F000958B
:1008A0001095031B130B08950091AE000430A1F1C5
:1008B000B0918D00B15008F010C0B0916100B093BC
:1008C0006300209277002092780020927900209295
:1008D0007A0020927B006F7B1FC06090AE00606446
:1008E000B0916100B093620008E317EC20917300AF
:1008F0003091740036952795B62DBA9541F036950E
:100900002795B62DBA95BA9511F0369527958DDFB6
:100910000093770010937800089566FF1BC0009144
:100920007700B09162000B1B10917800120928F437
:100930000038BFEF1B0740F009C00F37120508F45D
:1009400005C00FE710E002C000E81FEF00937C0035
:1009500010937D00089566FF39C000917C00B0912E
:1009600079000B0F10917D00B0917A001B1F20E0E1
:1009700030917D0033230AF42A95B0917B002B1F20
:100980001AF4203F40F00AC02F3008F407C00FEFE0
:100990001FEF2FE003C000E010E020EF3091630074
:1009A000B09192003B1718F4332331F009C0B09195
:1009B0007D00BB235AF004C0B0917D00BB2332F40C
:1009C0000093790010937A0020937B00089566FFCE
:1009D0002FC02091CD0000917C00000F10917D0070
:1009E000111F40DF11232AF40038BFEF1B0740F02E
:1009F00009C00F37120508F405C00FE710E002C068
:100A000000E81FEF002352F0B0916200B01B0B2FE3
:100A100018F0013008F00AC001E008C000950F5F2F
:100A2000B09162000B0F08F001C00FEF00937E0041
:100A3000089566FF2DC02091CE0000917A0010919C
:100A40007B0010DF11232AF40130BFEF1B0740F0B9
:100A500009C00F3F120508F405C00FEF10E002C0F7
:100A600001E01FEF112352F0B0917E00B01B0B2F5D
:100A700018F0013008F00AC000E008C000950F5FD0
:100A8000B0917E000B0F08F001C00FEF00936300E0
:100A900008950FEF677FB72FB670E9F46860B091E3
:100AA0007400B83008F0677FB0917400A1F00FEFC8
:100AB00010917400ACDEF894B09170000B9F112D72
:100AC000002D7894112309F00FEFB09195000B17CA
:100AD00010F40091950000939400089542D374FFA0
:100AE000B2E074FDB1E0B7B9B6B1B068B064B6B900
:100AF00038DE74FFB2E074FDB1E0B7B9B6B1B068EA
:100B0000B064B6B9B6B1B6FDFDCF04B115B1B6B19A
:100B1000BF77B6B979D324E72093A30030E03093B0
:100B2000A400732E7694622E6694620E731E262D98
:100B3000372D0217130778F08090A300B4E7B80DA3
:100B4000B093A3008090A400B0E0B81DB093A400BF
:100B5000260D371DEECF8090A3009090A400109139
:100B6000A40016950091A300079516950795B091DE
:100B7000A300B00FB093A100B091A400B11FB09337
:100B8000A20023E0169507952A95E1F72091AF0082
:100B90002A9529F42092A3002092A4000AC02A9545
:100BA00021F0800E911E2A95E1F78092A300909289
:100BB000A40008952091AF00B6B1B6FDFBCF04B1FB
:100BC00015B1B6B1BF77B6B9B091A500B395B093E2
:100BD000A500B83060F12092A500B091CC00BB23F5
:100BE00021F1112329F0B091A600BF3F61F009C0A7
:100BF000B091A6000B1739F020F4BB2321F0BA9571
:100C000002C0B395E1F300919200B093A600B8380A
:100C100050F400ECBD3738F400E8B23720F400E4BB
:100C2000B73608F400E0009392007F7E08952130EB
:100C300099F00F3FB3E01B0778F4B091A3000B17B6
:100C4000B091A4001B0740F4B0919200BB23A9F01F
:100C5000BA95B093920011C0B0919200BF3F69F075
:100C6000B395B0939200B091B400B33031F4B09129
:100C70009200BC5F10F4B093920000919200B0918A
:100C80006300B01B10F400916300B09193000B1748
:100C900050F000919300B0919300BF3F21F0B091CC
:100CA0009300B0939200B091AE00B43009F406C046
:100CB000B09194000B1708F00B2F502EB091A500A7
:100CC000B73009F47061089502E3F894B091D00050
:100CD0000B9F012D000C001F7894B09192000B1710
:100CE00010F0009192000093610000936300502E79
:100CF00000939500089520927300B8E0B0937400BB
:100D000008952091800030918100F8940CB51DB5B4
:100D1000200F311F3BBD2ABD6160B0E1B8BF7894A0
:100D20002091710030917200009371001093720055
:100D3000021B130B2091730030917400622E732EEE
:100D4000B4E08B2EB2E09B2EB0917400B43010F062
:100D50008A949A94B83010F08A949A94769467940E
:100D60008A94E1F726193709992021F016950795FD
:100D70009A94E1F7200F311F209373003093740091
:100D800008F00895BFEFB0937300B0937400089516
:100D90002091820030918300F8940CB51DB5020FAC
:100DA000131F1BBD0ABD6160B0E1B8BF7894089500
:100DB00060FDFECFEDDF0895B091BE0000916E00A2
:100DC000023808F0B395003A08F0B395B63008F051
:100DD000B5E09B2EBCE08B2EB0917400B33030F4A4
:100DE0008394839482FF02C083948394B23030F45E
:100DF0008394839482FF02C08394839471FF03C021
:100E0000B3E09B2E822C109174000091730024E0BB
:100E1000169507952A95E1F70819120928F0B02FC1
:100E2000B250B12FB20910F402E010E0312F202FA0
:100E3000712E602E76946794B92DB330E9F0B0FD31
:100E400005C0060D171D262D372D06C0000F111FDA
:100E50000250120922E030E0B92DB33068F020933F
:100E6000840030938500009380001093810060928D
:100E7000820070928300089500938400109385008F
:100E800020938000309381006092820070928300F2
:100E9000089560FDFECF20918200220F30918300E3
:100EA000331FB72FB67021F020917300309174007A
:100EB000F8940CB51DB5020F131F1BBD0ABD616070
:100EC000B0E1B8BF7894089560612092760020E088
:100ED00004C060612092760020E2B72FB67009F05E
:100EE0006F7E789460FD05C0B0917600BB2309F059
:100EF000089501E063FF0AC0B0917400B33008F0B8
:100F000002E0B0917400B63008F003E071FF01C058
:100F100006E060FD06C0B0917600BB2311F0789426
:100F200008951AE083FF1AE0789400000000F89416
:100F300062FD03C014E183FF14E171FF01C018E7F3
:100F4000B4B530919900B31BB10B18F3B091760092
:100F5000B395B0937600B5E03B2F6B2E722CB8B1F1
:100F6000B072B21709F073943A95C9F77394761476
:100F700088F464FFB2CF6F7E3CB56DB4709073009F
:100F800080907400370D681C6BBC3ABD6160B0E1A5
:100F9000B8BFA3CF64FDA1CF0A9509F0BACF78946A
:100FA000089571FF0AC0B0916D00B395B0936D00C4
:100FB00060FD0CC020926D0009C060FD07C064FD9B
:100FC00005C067FD03C0BF91BF9195C408952091EE
:100FD000840030918500F8940CB51DB5020F131FE5
:100FE0001BBD0ABD6160B0E1B8BF78940895EFDF22
:100FF00000E063FF03C064FF01C001E0F8941091BA
:101000006E00B7E01B9F212D102D7894200F2695A0
:101010001795269517952695179510936E001837F6
:1010200018F4B8E7B0936E0000916E00B0916F00B5
:101030000B1720F060629598AC98C09860FDFECFC9
:101040000895F894949AAD9AAB9A82FF07C0E2E0B3
:10105000F1E073FF03C0B5E0BA95F1F7B091740009
:10106000BC7F81F0552021F095FF959A95FDC09A9F
:10107000B6E0BA95F1F795FF959895FDC098B5E063
:10108000BA95F1F795FF949895FDAB98B2E0B093BF
:101090007500ABC0F89495FFC09895FD959882FFB8
:1010A0000DC0E2EFF0E073FF0BC0AD9A95FFAB9A75
:1010B00095FD949AB5E0BA95F1F702C0ECEAF0E03C
:1010C00062FF03C0552009F0AC9AB3E0B0937500FD
:1010D0008CC0F894949AAD9AAB9A82FF07C0E2EE66
:1010E000F0E073FF03C0B5E0BA95F1F7B09174007A
:1010F000BC7F81F0552021F095FFC09A95FD959A0F
:10110000B6E0BA95F1F795FFC09895FD9598B5E0D2
:10111000BA95F1F795FFAB9895FD9498B4E0B0932C
:10112000750063C0F894AC9882FF0DC0E2EDF0E06A
:1011300073FF0BC095FF949A95FDAB9AAD9AB5E0FD
:10114000BA95F1F702C0E4EAF0E062FF06C055206C
:1011500021F095FF959A95FDC09AB5E0B093750082
:1011600044C0F894949AAD9AAB9A82FF07C0EFEB13
:10117000F0E073FF03C0B5E0BA95F1F7B0917400E9
:10118000BC7F51F0552009F0AC9AB6E0BA95F1F762
:10119000AC98B5E0BA95F1F7AD98B6E0B0937500AC
:1011A00024C0F89495FF959895FDC09882FF10C0D3
:1011B000E5E1F1E073FF0EC095FF949A95FDAB9ABF
:1011C00095FFAB9A95FD949AB5E0BA95F1F702C0F8
:1011D000E4EBF0E062FF06C0552021F095FFC09AD5
:1011E00095FD959AB1E0B093750067FF0AC00CD0E9
:1011F000B5E0BA95F1F7B5E0BA95F1F79498AD98E6
:10120000AB986F7D7894089523EA30E0F9019598C2
:10121000AC98C098949AAD9AAB9A6B7F0895ACEA5B
:10122000B0E009E00D9309E00D9304E00D9301E0B7
:101230000D9303E00D930FEF0D930BE00D9301E081
:101240000D9301E00D9301E00D93A8EBB0E001E0F8
:101250000D930FEF0D930D930FEF0D930D930D93D2
:1012600003E00D9306E00D930FEF0D930D9305E250
:101270000D9300ED0D9308E20D9300E50D9304E04E
:101280000D930DE00D9302E00D9300E00D930AE73E
:101290000D930FEF0D9301E00D9308952091BF0082
:1012A00009E011E0223011F405E011E0233011F4DF
:1012B00005E012E0243011F405E013E0253011F4CC
:1012C00009E017E0263011F400E010E000939F00E1
:1012D0001093A0002091B3008B7F233009F4846029
:1012E000777F233009F47860B091B400B33019F0FF
:1012F0009F7DB1FD90629F7BB091B500B1FD906480
:10130000B22FB23011F0886001C0877F0895ECE100
:10131000F0E00091AC000A95E00FF21DB491B0939B
:10132000CD000091AD000A95E00FF21DB491B0938D
:10133000CE006ADF0895EAE2F0E00091C7000A9566
:10134000E00FF21DB491B093CF005EDF0895E8E3A3
:10135000F0E00091B2000A95E00FF21DB491B09355
:10136000D00052DF08950895B091C8000FEF1CE03F
:10137000B23011F400EA1AE0B33011F402E815E0DB
:1013800000936F0010937000089508952091C2009B
:101390003091C30097FF02C020E03FEFB32FB21B94
:1013A0006B2EB25810F4B2E86B2E00E00395609EED
:1013B000B12DB058D8F30093A7000895F894E3E056
:1013C000F0E0B9E0B7BFB491B078C1F3F894A89554
:1013D000B1B5B861B1BDB0E0B1BDB4E0BEBFBFE56D
:1013E000BDBF12DFB0E0B8BBB1E1B7BBB8E2B5BB7F
:1013F000B8E3B4BBB0E1B2BBB0E3B1BB2224A0E020
:10140000B0E02D92AA31E9F7A0E6B0E00FEF2D92FF
:101410000A95E9F704DF8FD241DF79DF8CDF97DFB0
:10142000A2DFA2DFB2DFB2DF0091C4000093A80008
:10143000EBDEB2E0B3BFB2E0BEBDB2E0B5BDF89442
:101440009AD9A4D994D9A5D992D9A6D990D993D902
:1014500092D98FD9B1E5B8BFB9BFB0B7B860B0BF46
:10146000B6B1B460B6B97DD9789438DBB0E4BBBF0F
:10147000BB27B064BABF8D7F7ED9B1E0B09369005D
:10148000626025E0B0918C00BB2309F425E06BD9A4
:10149000B0918D00B230A8F3B92FBF7100918F00C9
:1014A00000938E00B0938F00B01759F72A9551F72B
:1014B0006D7F96FFB3E096FDB2E0B5BFBB27B06489
:1014C000BABF8D7F56D94FD902E0B92FBF7109F449
:1014D00000E0B0918D00B017B0F3F89457D956D909
:1014E00055D9789448D920927F00B091B400B33098
:1014F00009F472C038D9B091B800B13008F46CC0AA
:10150000B0916900B13008F467C0B92FBF71C1F064
:10151000B0918D00BF3F08F45FC0F89440D9789433
:1015200028D9B0918D00B130C0F7F8942FD91DD9CA
:101530002DD978941ED9B0918D00BF3FB0F3C4C2AD
:10154000B3E09B2E9068F89421DF789412D9F89438
:101550009F771CDF80908D00B0918D00BF3778940D
:1015600008F442C0FED8F8941AD978949A9451F7A6
:10157000B82DB550B093C300FED8F89409D277D2F5
:101580007894BAE09B2E9068F89400DF7894F1D8B4
:10159000F8949F77FBDE80908D00B0918D00BF376F
:1015A000789478F7DED8F894F1D8DFD8EFD878942B
:1015B0009A9449F7B82DBB5FB093C200DCD8F89479
:1015C000E7D164D27894D5D8F894E0DE7894B091DD
:1015D0008D00BF3FC0F378C200918D00B0917F00B5
:1015E0000B1710F000937F00C4D801E0B091B40055
:1015F000B35009F405E0B0918D00B01708F075CF35
:10160000F894CDD8CCD8CBD87894B5D820926900AE
:1016100020926A0020926B00B0916A00B395B0935B
:101620006A00BF3F69F5B0916B00B395B0936B0052
:10163000B091C60009E1BA9559F002E3BA9541F0BC
:101640000DE7BA9529F00AEFBA9511F020926B00D8
:10165000B0916B00B017A0F0B0916B00BA95B09349
:101660006B00B4EBB0936A00B091C500B093A800D2
:10167000F89495D87894B091C400B093A80079D824
:1016800074D8B0916600BB2321F4B92FBF7109F45F
:10169000F7CEB0918D00B63008F4BECFB091B40053
:1016A000B35009F066D8B0916600BB2309F4E8CEC8
:1016B000F894AADD209261002092620020926300DB
:1016C000522C7894B091B100B0939600209277009C
:1016D000209278002092790020927A0020927B005C
:1016E0002092A50060E070E020926E0004DBB8E07C
:1016F000B093A500706135D874FFB2E074FDB1E01D
:10170000B7B9B6B1B068B064B6B9B6B1B6FDFDCF81
:1017100004B115B1B6B1BF77B6B9112309F00FEF17
:101720000093A60047DAB8E0B093A50070618090FE
:10173000B300B2E0B093B300B1DD8092B300F8948F
:10174000BFEFB0939200C0DAB0916100B093920005
:10175000B0939300B09394007894B1E0B09361009B
:10176000B09363005B2EB0939B00B0919100B09357
:101770009A007160726020926D00F3DC12DDC1DAB4
:10178000BADA1ADB04C08ADD2092A5007F7E95FFBD
:10179000B6E095FDB0E0B7B99CDB03DC18DC84D87B
:1017A00026DC4FDCAEDA04DB07DB73DBB7E0B7B96E
:1017B0008BDBF7DB0CDCB1D86CD919DC6BDCA1DA84
:1017C000F7DAFADA66DB95FFB0E095FDB6E0B7B977
:1017D00080DBE7DBFCDBBFD80ADC7BDC92DAE8DA13
:1017E000EBDA57DB95FFB6E095FDB0E0B7B96CDBFF
:1017F000D8DBEDDBECD8FBDB95DC83DAD9DADCDA9D
:1018000048DBB7E0B7B965DBCCDBE1DB12D9EFDB56
:10181000A8DC77DACDDAD0DA3CDB95FFB0E095FDD5
:10182000B6E0B7B951DB74FFB2E074FDB1E0B7B90F
:10183000B6B1B068B064B6B9B4DBC9DBD8DBB1DC33
:1018400060DAB6DAB9DAB6D924DB71FF2EC067FDEB
:101850002CC0B0919500B0939200B0939300B091DA
:101860009100B0939A00B1E0B0939B0014E624E19C
:10187000B0916D00B11798F07D7F746020936C007B
:10188000B091B400B33051F4B0919500B093920090
:10189000BFEFB0939300B0E2B093940006C0B09154
:1018A0008D00B13008F073CF26C072FF10C067FD05
:1018B0000EC0B0916C00BA9511F47B7F64CFB093E9
:1018C0006C00B0918D00B13008F061CF14C0B091C0
:1018D0009000BA3F80F4B92FBF7121F4B091660037
:1018E000BB2349F0B091740000EF67FF01C000E630
:1018F000B01708F44CCFF89487DC8090B300B2E0C6
:10190000B093B300CBDC8092B300209261002092B0
:10191000620020926300522C209296007E7F789481
:1019200020D772DCB92FBF7129F4B0916600BB23B8
:1019300009F4A6CD6DCEEDE0F0E023D0053509F039
:101940001BC0EEE0F0E01DD00A3A09F015C03AE005
:10195000ACEAB0E0E3E0F0E014D00D9331963A95B4
:10196000D9F735E1A8EBB0E0EFE0F0E00AD00D9355
:1019700031963A95D9F702C052DC0AD0E4E2F0E0A1
:101980000895E199FECFEEBBFFBBE09A0DB3089539
:101990001ED03AE0ACEAB0E0E3E0F0E00D910FD009
:1019A00031963A95D9F735E1A8EBB0E0EFE0F0E0F9
:1019B0000D9105D031963A95D9F712D00895E19955
:1019C000FECF0DBBEEBBFFBBE29AE19A0895EDE0BE
:1019D000F0E00FEFF4DFEEE0F0E00FEFF0DF08955E
:1019E000EDE0F0E005E5EBDFEEE0F0E00AEAE7DF4E
:1019F00008953091A9000091AA00313011F40093AC
:101A0000AC00323011F40093AD00333011F4009388
:101A1000AE00343011F40093B000353011F400936F
:101A2000AF00363011F40093B200373011F4009358
:101A3000BE00383011F40093C700393011F4009320
:101A4000BF003A3011F40093B3003B3011F400931F
:101A5000C8003C3011F40093B4003D3011F4009301
:101A6000B500089525E087D62A95E9F708958ED622
:101A700090D692D694D679D689D68BD68DD68FD657
:101A800074D684D686D688D68AD6089588D684D643
:101A900080D67CD66AD683D67FD67BD677D665D6D7
:101AA0007ED67AD676D672D608958090A900909088
:101AB000AA006CD66BD66AD658D68A94D1F76FD660
:101AC00054D69A94E1F70895F894D1DF7894CADF58
:101AD000C9DFB1E0B093A900B1E0B093AA002092B1
:101AE000AB00F894E2DF7894B5E06B2E70908D0037
:101AF00042D6B0918D007B16C9F7B13018F0BF3FC8
:101B000040F107C076DFF89443DFB1DFB8E0B1BD44
:101B1000A9DF6A9459F7B091AB00B395B093AB00CD
:101B2000B33008F4DECF9EDFB091AA00B395B09336
:101B3000AA00F894B091A900BA95E6E4F0E0EB0FA2
:101B4000F21D049178940395B091AA00B01708F49F
:101B5000C6CF88DF87DFB091A900B395B093A90005
:101B6000B091A900BE3008F4B7CF59DBF89410DF6C
:061B7000B8E0B1BD77DF13
:00000001FF
